:020000040800F2
:1000000068050020D90000080D1200083D11000805
:1000100000000000000000000000000000000000E0
:10002000000000000000000000000000571200085F
:1000300000000000000000005512000859120008DE
:10004000EB000008EB000008EB000008EB000008E4
:10005000EB000008EB000008EB000008EB000008D4
:1000600000000000EB000008EB000008EB000008B7
:10007000EB000008EB00000800000000EB000008A7
:1000800000000000EB00000800000000000000007D
:10009000EB00000800000000EB000008EB00000887
:1000A000EB000008EB000008EB000008191800083E
:1000B00029180008EB000008000000000000000004
:1000C0000448854600F090F800480047FD1B0008F2
:1000D000C046C046680500200448804704480047E1
:1000E000FEE7FEE7FEE7FEE7FEE7FEE7D1120008C7
:1000F000C100000830B50B46014600202022012433
:1001000009E00D46D5409D4205D31D469540491B4B
:100110002546954040191546521E002DF1DC30BD94
:10012000F0B51FB40646002082B005464024019178
:1001300000901BE0019922460F46304600F042F83D
:10014000049A059B801A994110D3104619462246FD
:1001500000F028F8361A8F4101972246012000212D
:10016000009F00F01FF838184D4100902046641E93
:100170000028DFDC019B00982946324607B0F0BD1D
:10018000D2B201E00270401C491EFBD2704700222F
:10019000F6E710B513460A4604461946FFF7F0FF86
:1001A000204610BD10B5202A04DB0146203A9140BC
:1001B000002010BD914020239C1A0346E3401943C0
:1001C000904010BD10B5202A04DB0846203AD040EC
:1001D000002110BD0B46D340D0402024A21A9140EC
:1001E0000843194610BD0000064C0125064E05E0E7
:1001F000E36807CC2B430C3C98471034B442F7D348
:10020000FFF762FF681C0008881C0008704770B583
:100210000024014620314A79022A03D00421C16317
:10022000012418E0026813680E25AB4313600268CE
:1002300013685B085B001360436C1C2213400122AF
:1002400015469D40036C5D604A7100220A71816B06
:10025000002900D08847204670BD70B5044600F0E4
:10026000C7F80546601C00D0641C00F0C1F8401BB4
:10027000A042FAD370BD0000F8B500230124A2E02B
:1002800027469F403A4070D04D68022D01D0122D74
:1002900014D1DD08AD002D1800952D6A5E07AC461F
:1002A000F50E0F26AE46AE406546B543AC460E6928
:1002B0007546AE4065462E43009D2E624D68012D69
:1002C00005D0022D03D0112D01D0122D16D1856835
:1002D0000326AC465D00AE46AE406546B543AC462F
:1002E000CE687546AE4065462E43866046680D79F9
:1002F000BE43ED06ED0F9D403543456006685F0047
:100300000325BD40AE46AE430D79B446AE07B60FE9
:10031000BE4065462E430660C6687546AE438D688E
:10032000BD403543C5604D68ED004BD5294D6E6B22
:1003300026436E639E08284DB6007519AC46AD681D
:100340009E07360F0F27B740BD4305273F07B8422A
:1003500001D1002715E0214FB84201D1012710E05B
:100360001F4FB84202D102270BE02BE01D4FB842CD
:1003700001D1032705E01C4FB84201D1052700E059
:100380000627B7402F436546AF60184D2E684F686B
:100390009643FF0300D516432E606E684F68964360
:1003A000BF0300D516436E60AE684F689643FF02E8
:1003B00000D51643AE60EE684F689643BF0200D585
:1003C0001643EE605B1C0A681546DD4000D057E717
:1003D000F8BD000000100240000001400004005081
:1003E00000080050000C0050001C005000040140A8
:1003F00001480068704700001400002002480168AE
:10040000491C0160704700001400002010B5084826
:1004100000240168402211430160204600F00AF8E0
:10042000002801D0012401E000F01CF8204610BD96
:100430000020024070B5054609487D210024C9000E
:100440000068FFF757FE00F0F9FB002801D00124F7
:1004500004E000222946501E00F01AF8204670BD24
:10046000180000200448416B012211434163816B55
:10047000020411438163704700100240C106C90E97
:1004800001208840014908607047000000E100E059
:1004900010B500F0BDFE10BDF8B504460078544D0F
:1004A000800672D5524E0027403EB06BC00004D487
:1004B000B06BA9050843B06301274E480168C90520
:1004C00011D40168821511430160FFF791FF00907C
:1004D00005E0FFF78DFF0099401A642837D845489A
:1004E0000068C005F5D532680321090560680A4037
:1004F0000140914208D08103890F032904D131685A
:10050000890301D50120F8BD2A69032109040A40A5
:1005100022D0084090421FD0207880061CD5286940
:100520002A6988430121C9040A432A612A698A4346
:100530002A612861C0050FD5FFF75AFF009008E037
:10054000FFF756FF0099411A2B48814201D9032039
:10055000F8BD28698005F3D561688803800F0328FA
:1005600005D132680005824301400A4332602869A0
:10057000032261681204114008432861002F04D04F
:10058000B16B012000078143B1632078C00705D01B
:10059000E868A168800880000843E8602078800748
:1005A00005D5E8680C218843E1680843E8602078B5
:1005B000400706D5E868032189028843216908437A
:1005C000E8602078000706D5E8680321090388431E
:1005D00061690843E8602078000606D5E8680321D1
:1005E00089048843A1690843E8600020F8BD000041
:1005F000401002400070004088130000F8B50E461D
:1006000005007DD053480068C007C00FB0420AD231
:100610005048016849084900314301600068C0073B
:10062000C00FB04271D128784B4C800705D5E068E7
:10063000F0218843A9680843E0602878C00752D0B9
:100640006868022817D0032818D02168012818D01C
:100650008905002959DAE168890889000143E160C8
:10066000FFF7C6FE69680746022912D003291CD08D
:10067000012926D033E021688903EAE7216889014E
:10068000E7E74907E5E7FFF7B3FEC11B33488142BF
:1006900023D8E0680007800F0228F4D123E0FFF799
:1006A000A7FEC11B2D48814217D8E0680007800FC4
:1006B0000328F4D117E0FFF79BFEC11B27488142B6
:1006C0000BD8E0680007800F0128F4D10BE0FFF79A
:1006D0008FFEC11B2148814201D90320F8BDE0688B
:1006E0000007800FF3D11B480168C907C90FB14249
:1006F0000DD901684908490031430160006800E0F4
:1007000003E0C007C00FB04201D00120F8BD287837
:10071000400706D5E068072109028843E9680843D5
:10072000E0602878000707D5E0680721C902884300
:100730002969C9000843E06000F036F8E168084A1A
:100740000906090F515CC840064908600020FFF700
:1007500071FEF8BD00200240001002408813000026
:10076000441C000818000020044805490068C968B6
:10077000044A4905490F515CC840704718000020E1
:10078000001002405D1C0008044805490068C96863
:10079000044A8904490F515CC84070471800002082
:1007A000001002405D1C000810B5184AD1680C20EA
:1007B000084004280BD0082810D00C2810D050680E
:1007C0000004410F0120C003491C884010BD10687F
:1007D000C00601D50E4810BD0E4810BD0E4810BD14
:1007E00088020E4B000F185C0902D368890F491C60
:1007F000DB0301D5084A05E01268D20601D5044A98
:1008000000E0044A5043FFF775FC10BD00100240A1
:1008100000093D000024F40000127A00541C000876
:10082000FEB505007ED0FE4CE7680C20E668074068
:100830000120000406402878C00747D0082F05D0C3
:100840000C2F0AD101200004864206D120688003C3
:100850003CD568680028E5D038E0012069680004CC
:10086000814203D121680143216011E00523012267
:100870001B0492049942216802D111432160F1E7DF
:1008800081432160216801400091206890432060ED
:10089000686800280DD0FFF7ABFD009005E0FFF77A
:1008A000A7FD0099401A64287AD820688003F6D5FD
:1008B0000CE0FFF79DFD009005E0FFF799FD009922
:1008C000401A6428F0D820688003F6D4287880077E
:1008D00055D50923E868042F0DD00C2F01D1002E27
:1008E00009D000283BD02168994301432160FFF7DC
:1008F0007FFD064627E02168490701D5002891D0F1
:1009000061681F22120291432A6912021143616039
:100910002168994301432160FFF746FFE16809061A
:100920000A0F00E079E1BF49895CC840BE49086010
:100930000020FFF77FFD002872D120E0FFF758FD6F
:10094000801B0228B0D820684007F7D560681F21B7
:100950000902884329690902084360600FE02068A2
:10096000400840002060FFF743FD064604E0FFF723
:100970003FFD801B022897D820684007F7D42878CD
:10098000C0065FD5002F0CD0A869002849D0206888
:10099000FF21013108432060FFF72AFD06462DE0C4
:1009A000C0E02068800502D5A8690028A7D060684B
:1009B000072149038843296A084360606068297FEA
:1009C0000002000A090608436060286A410B012002
:1009D000C003491C8840E16809060A0F9149895CF7
:1009E000C840914908600020FFF724FD002817D176
:1009F00028E0FFF7FDFC801B0228A3D820688005B3
:100A0000F7D56068072149038843296A0843606075
:100A10006068297F0002000A09060843606011E04F
:100A2000E1E02168FF20013081432160FFF7E0FC15
:100A3000064604E0FFF7DCFC801B022872D8206821
:100A40008005F7D42878794E000724D568690028F6
:100A5000306910D0012108433061FFF7C9FC0090D4
:100A600005E0FFF7C5FC0099401A02285AD8306902
:100A70008007F6D50FE0400840003061FFF7B8FC72
:100A8000009005E0FFF7B4FC0099401A022849D80D
:100A900030698007F6D42878400765D50020029099
:100AA000A06BC00006D4A06B012109070843A06316
:100AB000012002905E480168C90511D401688215C1
:100AC00011430160FFF794FC009005E0FFF790FCF4
:100AD0000099401A642825D855480068C005F5D506
:100AE000FF20AA680130824203D13169014331619C
:100AF00011E001218902002A07D005231B029A4236
:100B000003D132690A433261EFE7326982433261CD
:100B1000306988433061A86800280FD0FFF768FC6F
:100B2000009007E05EE0FFF763FC0099411A41483E
:100B3000814257D830698005F5D50DE0FFF758FCA4
:100B4000009006E0FFF754FC0099411A39488142B1
:100B500048D830698005F5D40298002804D0A06BED
:100B6000012109078843A063686A002864D00C2F1C
:100B70003ED0012636060228206805D0B04320600A
:100B8000FFF736FC05462FE0B0432060FFF730FC4E
:100B9000074604E0FFF72CFCC01B022822D820687F
:100BA0008001F7D4E96AA86AE2680843296BFD234B
:100BB0001B049A4311430843E060206830432060DF
:100BC000FFF716FC054604E0FFF712FC401B022865
:100BD00008D820688001F7D52EE0FFF709FC401BFC
:100BE000022801D90320FEBD20688001F5D423E04E
:100BF0000128F8D0E06801210904AA6A0140914265
:100C00000BD10F218904EA6A0140914205D10321E9
:100C100089050840296B88420ED00120FEBD0000E6
:100C200000100240441C0008180000204010024040
:100C300000700040881300000020EFE7094910B55C
:100C4000401E884201D9012010BD074C606103217C
:100C5000081F00F0DDFA0020A061072020610020BD
:100C600010BD0000FFFFFF0000E000E0F0B502460D
:100C70002032137E012B15D00127177602235376DD
:100C800005686C68AB687026B4430E6849682643F3
:100C90008024A34319436E6000688160577600206A
:100CA0001076F0BD0220F0BD70B5040005D02546D9
:100CB0002035687E002802D006E0012070BD0020AB
:100CC0002876204600F00AF802206876211D206868
:100CD00000F028FB01206876002070BD0068044900
:100CE000884204D10348816B10221143816370470D
:100CF000001000400010024070477047F8B50268CD
:100D00000446D0691168936805072D0F5BD0DD0795
:100D1000ED0FFF2621360E402E4367D0C60706D0C2
:100D2000CE0504D501261662E26F3243E2678707DB
:100D300002220426002F06DADF0704D027683A6271
:100D4000E76F3743E767470706D5DB0704D023681B
:100D50001E62E36F1343E367020709D520220A40AE
:100D60002A4305D0236808221A62E36F1343E3671E
:100D7000E26F002A2FD0800606D5880604D5216EA2
:100D8000002901D020468847E06F2168896849061C
:100D900001D4000724D5204600F090FB206881682C
:100DA000490619D58168402291438160E06E002890
:100DB00012D020498163E06EFFF729FA00280AD09B
:100DC000E06E816B06E0850610D58D060ED5216E8E
:100DD0001CE020468847F8BD2046FFF78EFFF8BD8F
:100DE0002046FFF78AFF0020E067F8BDC50208D55E
:100DF0005B0206D50120000510622046FFF77CFF4C
:100E0000F8BD030605D50B0603D5616E0029E0D1B8
:100E1000F8BD4006FCD54806FAD5136820464021A7
:100E20008B431360202161670021616600F085F922
:100E3000F8BD0000A914000810B5040003D0606FCD
:100E4000002802D007E0012010BD002170200155CC
:100E5000204600F027F824206067206801684908D0
:100E600049000160204600F091FB0128ECD0606A47
:100E7000002802D0204600F081FA2068416809224B
:100E8000D20291434160206881682A2291438160A7
:100E900020680168012211430160204600F0D4FA65
:100EA00010BD0000F0B587B0044614216846FFF776
:100EB0006EF9244F266800212348012202230324CF
:100EC0000425BE421AD1466B97033E434663C66A69
:100ED0001643C662C06A02AE1040059060020090E0
:100EE000019332C6052069460007FFF7C5F90022C5
:100EF00011461B20FFF7CCFA1B201EE0134FBE4209
:100F00001DD1866B01277F043E438663C66A164364
:100F1000C662C06A02AEC007C00F05900C200090E8
:100F2000019332C6052069460007FFF7A5F90022A4
:100F300011461C20FFF7ACFA1C20FFF79FFA07B000
:100F4000F0BD0000003801400010024000440040A5
:100F5000F0B5836F202B54D100290AD0002A08D085
:100F60008568DC01A54206D10369002B03D1CB07BC
:100F700001D00120F0BD034660331E7C012E40D01D
:100F800001261E744165014640310A834A830022CE
:100F9000FF260266A54204D10569002D13D11A4D22
:100FA0000AE07F27002D09D001263607B5420CD173
:100FB0000569002D05D03F258D8307E00569002DCB
:100FC00001D08F8302E08E8300E08A83C2672221F2
:100FD000816701688D68012635438D608168A14273
:100FE00002D1016900290AD0084901661A74006813
:100FF0000168FF222132114301600020F0BD044945
:10100000F3E70220F0BD0000FF01000035150008E5
:10101000DD14000810B500680E49884219D10E4849
:101020000178012915D14178032912D1C1780279BB
:1010300009020A4C89182160427983791202D21878
:10104000A260C379007A1B021B1805A0636000F040
:10105000F3FB10BD004400402000002000000020F1
:101060002534642534642534640A0000FFB5044641
:10107000406F83B017460D4620285CD1002D0AD062
:10108000002F08D0A168C001814207D12069002843
:1010900004D1E80702D0012007B0F0BD204660303F
:1010A0000290007C012846D00298012101740020A2
:1010B000E06721206067FFF79BF9264640360190E4
:1010C000378277820120A1680003814202D1206922
:1010D000002802D02F46002511E000270FE0002253
:1010E0008021204600F066FB002815D1002F15D086
:1010F0002168387888627F1C708A401E7082708AEE
:10110000019B002806980090E9D10022402120464A
:1011100000F050FB002808D00320BDE72888216894
:10112000C005C00D8862AD1CE6E72020606702990B
:1011300000200874B0E70220AEE77047FEE7000029
:1011400008B50448C16A01221143C162C06A104057
:10115000009008BD001002401CB500240E48009409
:101160000C490194016007218460416001214461C0
:10117000C160FFF799FD002801D0FFF747F8009400
:10118000694605480194FFF771FD002801D0FFF77B
:101190003DF81CBD001000402C00002010B50C488C
:1011A0000A490160E1214902416000218160C1607A
:1011B00001618161C1610C22016242614162FFF7FC
:1011C0003BFE002801D0FFF721F810BD0038014098
:1011D0006800002010B50C480A4901604B21C90184
:1011E000416000218160C16001618161C1610C22A7
:1011F000016242614162FFF71FFE002801D0FFF744
:1012000005F810BD00440040E800002070470000D1
:101210008307FF22DB0E9A408907090E99400028B8
:101220000BDA0007000F0838830808489B001818DD
:10123000C36993430B43C3617047830804489B0011
:101240001B181868904308431860704700ED00E0D1
:1012500000E400E07047704710B5FFF7CFF810BD0D
:1012600030B599B034216846FEF791FF14210DA8DE
:10127000FEF78DFF1C2112A8FEF789FF13480168B5
:101280000322D2029143C214891801600220009007
:101290000024102009940125049003956846FFF767
:1012A000BFFA0F200D9080200F900E951094002112
:1012B00011940DA8FFF7A2F903201290149415942D
:1012C00012A8FFF7E9F819B030BD00000070004027
:1012D00010480168821511430160C1680E4A11402F
:1012E000C16001680D4A11400160816849084900E8
:1012F000816001680122920491430160C168FD226E
:1013000012049143C160002101610549C003886056
:1013100070470000001002400C40FF88F6FFF6FE08
:1013200000ED00E070B5026801239B07114C124DDF
:10133000984203D0A04201D0A84203D17026B24304
:101340004E683243984203D0A04201D0A84204D153
:1013500003231B029A43CB681A4380239A430B69E9
:101360001A4302608A68C262096881620121416190
:1013700070BD0000000801400014014010B5818CD0
:10138000C90707D001684A6801235B049A43836A4E
:101390001A434A60818C890707D501684A6801238E
:1013A0001B049A43C36A1A434A60818C490707D5D4
:1013B00001684A6801239B049A43036B1A434A60FD
:1013C000818C090707D501684A680123DB039A432A
:1013D000436B1A434A60818CC90607D5026891683D
:1013E00001231B039943836B19439160818C890608
:1013F00007D501688A6801235B039A43C36B1A43CC
:101400008A60818C490612D503685A680121090552
:10141000046C8A4322435A60026C8A4207D10268F4
:10142000516803235B059943436C19435160818CD8
:10143000090607D501684A680123DB04806C9A43DA
:1014400002434A6010BD0000F8B500260446C66796
:10145000FEF7CEFF054620680068124F000709D549
:1014600001212B46002249052046009700F0A2F9F1
:1014700000280DD12068006840070BD501212B46BC
:10148000002289052046009700F094F9002801D039
:101490000320F8BD20206067A06760342674002018
:1014A000F8BD0000FFFFFF0110B5806A0022014671
:1014B00040314A834A82FFF720FC10BD01680A6868
:1014C000FF2321339A430A6001688A685208520058
:1014D0008A602021816700210166704710B50146AE
:1014E00040318B8B846F0268222C04D090690821D4
:1014F0000843906110BD526A446D1A402280426DCB
:10150000921C42654A8B521E4A83498B0029F1D1B5
:1015100001680A68FF2321339A430A6001688A68D8
:10152000520852008A602021816700210166FFF77E
:1015300071FD10BD10B5014640318B8B846F026880
:10154000222C04D0906908210843906110BD526A92
:101550001A40436D1A70426D521C42654A8B521EEE
:101560004A83498B0029F1D101680A68FF2321339E
:101570009A430A6001688A68520852008A602021F2
:10158000816700210166FFF745FD10BDF8B50446EF
:101590002669A268E76932436669102000253E4348
:1015A0002368324378491E68784F3E4016431E60D8
:1015B00023685A6803263603B243E66832435A600A
:1015C0002368A2698B4201D0266A32439E680B27AA
:1015D0003F02BE4316439E606D4E23686D4AB34280
:1015E0000CD1D2689207920F06D0012A38D0022A75
:1015F00034D0032A20D11EE001201DE0664EB34204
:101600000AD1D2680C26324026D0042A28D0082AD3
:1016100024D00C2A10D10EE08B420DD1D6680322C3
:101620009202164018D001229202B61A18D0B61AA9
:1016300014D0964200D10820564A0126403A574F0E
:10164000F6038B4236D100280CD002280DD0042896
:1016500012D008281FD11CE00020EDE70220EBE7A4
:101660000420E9E7FFF780F808E01068C00601D51C
:10167000384605E04A4803E0FFF796F8002873D0A3
:10168000626851005118814205D81103814202D38A
:1016900003E03046F4E7012566E0010E060250083B
:1016A000002330185941FEF73BFD03210902411A7E
:1016B0003C4A55E0E169B14232D1030000F0CCF878
:1016C00009070A0D06250606062B0600E3E7FFF7C5
:1016D0004BF81CE0FFF758F819E010686168C00685
:1016E00002D54808304A01E0304A48088018FEF721
:1016F00001FD80B201462E4A10399142CBD8511CCF
:1017000001400007400F08432CE0FFF74DF86168E7
:1017100040004A08EAE76168012248081204E5E748
:10172000030000F099F809070A0D06260606062CA4
:101730000600B0E7FFF718F81DE0FFF725F81AE0FC
:1017400010686168C00602D54808C01902E0144854
:101750004A081018FEF7CEFC80B20146144A103930
:10176000914298D82168C8600020206660662846AB
:10177000F8BDFFF719F861684A088018EAE7616860
:1017800048088019E6E7000000480040F369FFEFD1
:1017900000380140401002400044004000093D0074
:1017A0000024F400FFFC0F0000127A000048E8015A
:1017B000EFFF0000FFB581B017460E4604460A9DB4
:1017C00009E0681C07D0FEF713FE0499401AA842EE
:1017D0000CD8002D0AD02068C1693046884318D043
:1017E0000020B842EDD0002005B0F0BD20680168AF
:1017F000FF22A132914301602068816849084900B5
:10180000816020206067A06700206034207403207E
:10181000EAE70120E5E7000010B50248FFF76EFA9D
:1018200010BD00006800002010B50248FFF766FAFE
:1018300010BD0000E80000200FB410B503A9044B50
:10184000044A029800F024F810BC08BC04B0184701
:10185000E11B00081C00002030B47446641E25788B
:10186000641CAB4200D21D46635D5B00E31830BCD4
:10187000184702E008C8121F08C1002AFAD17047B1
:101880007047002001E001C1121F002AFBD1704700
:10189000FFB58FB00546002606E025280AD0129A2B
:1018A000119990476D1C761C28780028F5D1304698
:1018B00013B0F0BD002402940121B54A009400E069
:1018C00004436D1C2B780846203B98401042F7D10A
:1018D00028782A280ED00222287801463039092992
:1018E00016D802990A2359433039401814436D1C05
:1018F0000290F1E7109802C802911090002904DAD2
:1019000001204003044348420290022004436D1C1E
:1019100028782E2817D10420044368786D1C2A28C3
:101920000CD110986D1C02C8009110900BE000992A
:101930000A225143303940186D1C00902878014626
:1019400030390929F3D928786C2810D006DC4C28C6
:101950001AD068280ED06A2817D104E0742813D052
:101960007A2812D110E00120400504430CE0012147
:10197000090501E0032109050C436978814203D17F
:101980000120000524186D1C6D1C2878692874D06E
:1019900006DC00288BD0632827D0642806D16CE0B1
:1019A0006E2808D073282CD0752878D0129A1199F7
:1019B0009047761C5FE06002400F022809D00328A0
:1019C0000DD00428109801680DD00E60001D1090F5
:1019D00051E01098F21701680E604A60F6E710981F
:1019E00001680E80F2E70E70F0E710986A46017801
:1019F0001173001D10900020507303A80190012066
:101A000005E0109802C8019110900020C0436107C2
:101A10000CD5002700E07F1C00998F420FDA874227
:101A2000F9DB0199C95D0029F5D108E0002700E044
:101A30007F1C8742FCDB0199C95D0029F8D102981F
:101A40002146C01B0290129B119A00F0B3F8801936
:101A5000C61907E0019801990078491C0191129A72
:101A6000119990477F1EF5D22146129B119A029838
:101A700000F090F886196D1C16E70A200190109965
:101A800001C910916102490F032900D100B2042954
:101A900000D140B2002803DA40422D2103E00DE0DE
:101AA000210504D52B216A461173012103E0E107CA
:101AB00011D02021F7E70CAF0C9114E00A2001901F
:101AC000109901C910916102490F032900D180B218
:101AD000042900D1C0B20021EDE70199FEF70AFB0D
:101AE00030317F1E39700028F7D104A8C01B203088
:101AF0000190600704D5012000048443009801E0B0
:101B0000012000900199884201DD401A00E0002088
:101B1000411800900C9809180298401A0290E003AE
:101B200006D42146129B119A029800F043F88619B8
:101B300000200D9008E003A9085C129A11999047C3
:101B40000D98401C761C0D900C998842F3DBE00345
:101B50000CD52146129B119A029800F02BF8861999
:101B600004E0129A302011999047761C0099481E83
:101B700000900029F5DC05E03878129A7F1C119955
:101B80009047761C0199481E01900029F4DC6BE710
:101B900009280100F8B5044600251E4617468804AA
:101BA00004D405E039462020B0476D1C641EF9D5E9
:101BB0002846F8BDFFB50446002581B01E46C8037F
:101BC00001D5302700E02027880404D505E03846F9
:101BD0000399B0476D1C641EF9D5284605B0F0BDC9
:101BE00001B5044B012269460348FFF73FFA00980C
:101BF00008BD0000FFFF000068000020FEF706FCA3
:101C0000FFF72EFBFFF79CFAFFF7C8FAFFF7A4FADD
:101C1000FFF7E0FA074C3223082207490748FFF78D
:101C200025FA0B2206490548FFF792F92046FEF7F0
:101C300014FBF0E7102700000C000020E800002053
:101C4000200000200000000000000000010203044A
:101C500006070809030406080C10182030000000CD
:101C60000001020304000000881C0008000000209E
:101C70002000000072180008A81C000820000020A6
:101C80004805000082180008000000000000000065
:101C90000000000001030000000305CB000000006D
:081CA00000002000000000001C
:04000005080000C12E
:00000001FF
